:100000000C9464000C94980A0C94C50A0C948C000F
:100010000C948C000C948C000C948C000C94F107C4
:100020000C948C000C948C000C948C000C948C0020
:100030000C948C000C948C000C948C000C948C0010
:100040000C94A9130C948C000C9419030C948C0040
:100050000C948C000C948C000C948C000C948C00F0
:100060000C94C9180C948C00020000000024002796
:10007000002A0000000000250028002B00000000DE
:1000800000230026002900040404040404040402DC
:100090000202020202030303030303010204081025
:1000A00020408001020408102001020408102000F2
:1000B0000000070002010000030406000000000029
:1000C00000000000A604641711241FBECFEFD8E083
:1000D000DEBFCDBF12E0A0E0B1E0EAEEFAE402C07C
:1000E00005900D92AA3BB107D9F714E0AAEBB2E054
:1000F00001C01D92A934B107E1F710E0C8ECD0E0CF
:1001000004C02297FE010E94D521C43CD107C9F743
:100110000E94F0010C9473250C9400000F931F9320
:1001200060ED77E080E090E00E94311408E513E094
:10013000C80160E071E00E94170560ED77E080E0A3
:1001400090E00E943114C8010E9487041F910F9112
:1001500008950F931F9386E060E00E94211508E543
:1001600013E0C80140E056E960E070E00E94AA0395
:10017000C8016BE071E00E941705C80169E171E0F8
:100180000E941705C80163E371E00E941705C801CA
:1001900061E471E00E941705C8016FE471E00E94FC
:1001A0001705C80160E671E00E9417050E948E00E5
:1001B0001F910F910895F894FFCF84E061E00E94B1
:1001C000741583E061E00E9474158AE090E00E945B
:1001D000571484E060E00E9474158AE090E00E9469
:1001E000571483E060E00E9474158AE090E00E945A
:1001F0005714089584E060E00E9474158AE090E04E
:100200000E94571483E061E00E9474158AE090E038
:100210000E94571484E061E00E94741508958AE0FA
:1002200090E00E94571483E060E00E94741584E11E
:1002300090E00E94571483E061E00E9474158AE008
:1002400090E00E94571408950F931F938AE090E066
:100250000E94571400E017E084E00E94A915682F5F
:1002600090E0012E02C0880F991F0A94E2F7082B34
:100270008CE00E9474150E940F01115068F70E94D3
:100280000F01802F1F910F9108958AE090E00E9446
:10029000571483E061E00E94741584E190E00E94AD
:1002A000571483E060E00E9474158AE090E00E9499
:1002B000571408951F93CF93DF9317E0C82FD0E012
:1002C000BE01012E02C0759567950A94E2F7617030
:1002D00084E00E9474150E944501115088F784E063
:1002E00061E00E9474150E944501DF91CF911F913A
:1002F000089584E060E00E94211583E061E00E949F
:100300007415089584E061E00E94211583E061E0A6
:100310000E9474150895EF92FF920F931F9380919E
:10032000C502879588278795F090C602FF0CFF0CC1
:10033000FF0CF82A8091C702F82A8091C9028295A1
:10034000880F807E0091CA02000F000F000F082B5B
:100350008091C802082B9091CB0297959927979589
:100360008091CF028295807F892B9091D102892B39
:100370009091D302990F990F990F982BE090CE028C
:10038000EE0CE92A9091CC02979599279795809148
:10039000CD028295880F880F807C892B9091D202A4
:1003A000892B1091D002110F110F182B0E9482017E
:1003B0000E94DD0088EC0E945A018F2D0E945A0194
:1003C000802F0E945A018E2D0E945A01812F0E9477
:1003D0005A010E94FA001F910F91FF90EF9008952B
:1003E0008F929F92AF92BF92CF92DF92EF92FF9245
:1003F0000F931F93DF93CF93CDB7DEB727970FB639
:10040000F894DEBF0FBECDBF0E94611488ED93E06B
:100410000E94D91785E061E00E94211585E060E027
:100420000E9474150E94A90082E060E00E942115DC
:1004300083E061E00E94211586E060E00E942115C2
:100440008CE061E00E9421158DE061E00E942115A1
:100450008DE061E00E94741585E061E00E947415F2
:100460006AEF70E080E090E00E9431140E948B01FE
:10047000AAEFEA2EF12C4E010894811C911CF4E0A5
:10048000AF2EB12CAC0EBD1EE2E0CE2ED12CCC0E88
:10049000DD1E82E00E94A915019709F0BCC08CE026
:1004A00061E00E9474158DE060E00E9474150E9466
:1004B00082010E94DD0089EC0E945A0182E00E94C4
:1004C000A915892B09F0A7C08DE061E00E94741581
:1004D0000E9479010BEB12E00E942401F801819344
:1004E0008F01F2E0053C1F07B9F70E9482010E94CC
:1004F000FA008091BB0289832091BD0230E040E088
:1005000050E0542F432F322F22278091BE0290E0DB
:10051000A0E0B0E0282B392B4A2B5B2B8091BC024A
:1005200090E0A0E0B0E087709070A070B070DC0147
:1005300099278827282B392B4A2B5B2B2C833D832B
:100540004E835F832091C0022295269526952370C5
:1005500030E08091BF0290E0880F991F880F991FAB
:10056000282B392B3B832A8317C088E593E00E9410
:100570006304823029F0833061F0813069F404C073
:100580002AEFE22EF12C08C098EEE92E93E0F92E26
:1005900003C082E3E82EF12C88E593E00E94380442
:1005A0001816190614F386E00E94A9152091BA02C4
:1005B000892B59F1222319F481E08093BA0288E54E
:1005C00093E063E771E042E050E00E94F80488E5C0
:1005D00093E062E771E041E050E00E94F80488E5B2
:1005E00093E0B40141E050E00E94F80488E593E014
:1005F000B50144E050E00E94F80488E593E0B601BC
:1006000042E050E00E94F80406C0222321F00E943C
:100610008E001092BA02B70180E090E00E9431147F
:100620008CE060E00E9474158DE060E00E9474151B
:1006300030CF1F920F920FB60F9211242F933F933A
:100640004F938F939F93EF93FF934091C600E09158
:100650005403F091550331969F012F7730703197F5
:1006600080915603909157032817390739F0EC52BF
:10067000FD4F40833093550320935403FF91EF9136
:100680009F918F914F913F912F910F900FBE0F909F
:100690001F9018958F92AF92CF92DF92EF92FF92B8
:1006A0000F931F93DF93CF93CDB7DEB7FC0189E79C
:1006B00091E091838083738362835583448337837E
:1006C000268311870087F386E286D586C486A686B0
:1006D00087868D85808B8E85818B8F85828BCF9150
:1006E000DF911F910F91FF90EF90DF90CF90AF902F
:1006F0008F9008958F92AF92CF92DF92EF92FF92F8
:100700000F931F93DF93CF93CDB7DEB7FC0189E73B
:1007100091E091838083738362835583448337831D
:10072000268311870087F386E286D586C486A6864F
:1007300087868D85808B8E85818B8F85828BCF91EF
:10074000DF911F910F91FF90EF90DF90CF90AF90CE
:100750008F900895EF92FF920F931F938C019A014F
:10076000AB01DC011896ED91FC91199791E0E92E0F
:10077000F12CC70152960C9002C0880F991F0A9461
:10078000E2F7808360E874E88EE190E00E945F21E8
:100790002150304040405040569547953795279519
:1007A000D8011496ED91FC91159730831696ED9132
:1007B000FC91179720831A96ED91FC911B9720814D
:1007C000C7011E960C901E9702C0880F991F0A94AD
:1007D000E2F7282B20831A96ED91FC911B9720813C
:1007E000C7011F960C901F9702C0880F991F0A948B
:1007F000E2F7282B20831A96ED91FC911B978081BC
:1008000050960C9002C0EE0CFF1C0A94E2F78E2961
:1008100080831F910F91FF90EF900895FC01A285B6
:10082000B3854C9121E030E0C901068402C0880FF5
:10083000991F0A94E2F7809584238C93A285B3854F
:100840004C91C901078402C0880F991F0A94E2F7EE
:10085000809584238C93A285B3858C91008802C0F7
:10086000220F331F0A94E2F7209528232C93089532
:10087000DC011296ED91FC911397E058FF4F219106
:10088000319180819181281B390B2F773070C901FC
:100890000895DC011296ED91FC911397EE57FF4FEE
:1008A0002081318192918291E058F0408217930724
:1008B00019F42FEF3FEF05C0E20FF31F8081282FBF
:1008C00030E0C9010895DC011296ED91FC91139777
:1008D000DF01AE57BF4F2D913C911197E058FF4F6C
:1008E00080819181E058F0408217930719F42FEF2F
:1008F0003FEF0BC0E20FF31F80812F5F3F4F2F7739
:1009000030702D933C93282F30E0C9010895DC010D
:100910001296ED91FC911397EE57FF4F80819181D4
:10092000929382930895FC01A085B18521898C91D1
:1009300090E0022E02C0959587950A94E2F780FF19
:10094000F6CF0484F585E02D6083089589E791E072
:10095000909359038093580384ED92E090935B0346
:1009600080935A0385EC90E090935D0380935C0341
:1009700084EC90E090935F0380935E0380EC90E0C2
:10098000909361038093600381EC90E09093630304
:100990008093620386EC90E09093650380936403F8
:1009A00084E08093660383E08093670387E080930D
:1009B000680385E08093690381E080936A0308956A
:1009C0000F931F93CF93DF938C01EB0109C0219606
:1009D000D801ED91FC910190F081E02DC8010995BD
:1009E00068816623A1F7DF91CF911F910F91089540
:1009F000EF92FF920F931F93CF93DF938C017B01B4
:100A0000EA010CC0D7016D917D01D801ED91FC91F7
:100A10000190F081E02DC80109952197209791F769
:100A2000DF91CF911F910F91FF90EF900895DC011E
:100A3000ED91FC910280F381E02D09950895CF920C
:100A4000DF92EF92FF920F931F93CF93DF936C018E
:100A50007B01C0E0D0E00EC0D601ED91FC91008199
:100A60001181C701BE010E94B90B682FC601F801B0
:100A700009952196F70184819581C817D90760F3FC
:100A8000DF91CF911F910F91FF90EF90DF90CF906A
:100A900008952F923F924F925F926F927F928F9222
:100AA0009F92AF92BF92CF92DF92EF92FF920F93FD
:100AB0001F93DF93CF93CDB7DEB7A0970FB6F8940F
:100AC000DEBF0FBECDBF1C016A017B014115510580
:100AD0006105710549F440E350E060E070E020E01A
:100AE00030E00E94150656C0882499245401422EF5
:100AF00055246624772401E010E00C0F1D1F080D1B
:100B0000191DC701B601A30192010E945F21F801DE
:100B100060830894811C911CA11CB11CC701B60103
:100B2000A30192010E945F21C901DA016C017D01DC
:100B3000C114D104E104F104F1F681E0E82EF12CB6
:100B4000EC0EFD1EE80CF91C3E010894611C711CA2
:100B5000D501C4010197A109B1096C01C818D908D0
:100B600016C0F601EE0DFF1D40814A3010F4405DC5
:100B700001C0495C552747FD5095652F752FC10170
:100B800020E030E00E9415060894E108F1086E1498
:100B90007F0439F7A0960FB6F894DEBF0FBECDBF25
:100BA000CF91DF911F910F91FF90EF90DF90CF9049
:100BB000BF90AF909F908F907F906F905F904F907D
:100BC0003F902F900895DC012115310541F4ED91FE
:100BD000FC910190F081E02D642F099508950E9409
:100BE00049050895EF92FF920F931F939A017B019D
:100BF00000E010E0B801A7010E94E3051F910F91EA
:100C0000FF90EF900895EF92FF920F931F939A0138
:100C1000E62EFF2400E010E0B801A7010E94E305E2
:100C20001F910F91FF90EF900895EF92FF920F9315
:100C30001F93CF93DF93EC017A018B0121153105CE
:100C400041F4E881F9810190F081E02D642F09954C
:100C50001BC02A303105B1F477FF10C04DE250E0DF
:100C600060E070E020E030E00E94150610950095ED
:100C7000F094E094E11CF11C011D111DCE01B8019E
:100C8000A7012AE00E944905DF91CF911F910F91A2
:100C9000FF90EF900895EF92FF920F931F937B01C7
:100CA0009A010027F7FC0095102FB801A7010E94B8
:100CB00015061F910F91FF90EF900895EF92FF920C
:100CC0000F931F93E62E9A01FF24E7FCF0940F2D5B
:100CD0001F2DB801A7010E9415061F910F91FF90CB
:100CE000EF9008950F931F938C014DE050E060E06A
:100CF00070E020E030E00E941506C8014AE050E0B4
:100D000060E070E020E030E00E9415061F910F9136
:100D100008950F931F938C010E94E305C8010E9460
:100D200072061F910F910895CF92DF92EF92FF927A
:100D30000F931F938C019A016B01EE24FF24B701DE
:100D4000A6010E94E305C8010E9472061F910F913F
:100D5000FF90EF90DF90CF900895CF92DF92EF92C7
:100D6000FF920F931F938C019A01C62EDD24EE246F
:100D7000FF24B701A6010E94E305C8010E94720684
:100D80001F910F91FF90EF90DF90CF9008950F93F8
:100D90001F938C010E941705C8010E9472061F91C3
:100DA0000F9108950F931F938C010E941F05C80196
:100DB0000E9472061F910F9108950F931F938C014B
:100DC0000E941506C8010E9472061F910F91089596
:100DD000CF92DF92EF92FF920F931F938C016B01E2
:100DE0009A01EE24D7FCE094FE2CB701A6010E94E4
:100DF0001506C8010E9472061F910F91FF90EF9097
:100E0000DF90CF900895CF92DF92EF92FF920F93F1
:100E10001F938C01C62E9A01DD24C7FCD094ED2CC3
:100E2000FD2CB701A6010E941506C8010E9472069A
:100E30001F910F91FF90EF90DF90CF9008959F92B8
:100E4000AF92BF92CF92DF92EF92FF920F931F93D8
:100E5000CF93DF93EC017A018B01922ECB01BA0183
:100E600020E030E040E050E00E94F01D88236CF468
:100E7000CE014DE250E060E070E020E030E00E9402
:100E8000150617FB109517F9109520E030E040E0AB
:100E90005FE3AA240BC0CA01B90120E030E040E2C0
:100EA00051E40E94141D9B01AC01A394A91498F372
:100EB000C801B7010E94ED1B5B016C010E94441A3E
:100EC0007B018C01CE01B801A7012AE030E00E942D
:100ED000E305992029F0CE0169E971E00E94170528
:100EE000C801B7010E94D21E9B01AC01C601B50129
:100EF0000E94BC1B22C020E030E040E251E40E948E
:100F00001A1C7B018C010E947E1E5B016C01CC24AB
:100F1000B7FCC094DC2CCE01B601A5012AE030E07C
:100F20000E941506C601B5010E94201E9B01AC015E
:100F3000C801B7010E94BC1B9A949920E1F6DF9189
:100F4000CF911F910F91FF90EF90DF90CF90BF90C6
:100F5000AF909F9008950E941F0708950F931F93CD
:100F60008C010E941F07C8010E9472061F910F91F9
:100F70000895813041F0813018F08230D1F409C0F9
:100F800010926E00089580916F008D7F80936F00A6
:100F90000895809170008D7F8093700081E0809330
:100FA000B0008091B100887F84608093B10010927E
:100FB000B30008951F93182F8091A501811711F098
:100FC0009FEF06C0E8E6F0E094918FEF8093A501D3
:100FD000892F0E94B907812F60E00E9474151F912C
:100FE00008951F920F920FB60F9211242F933F93E3
:100FF0004F935F936F937F938F939F93AF93BF9321
:10100000EF93FF938091790390917A03A0917B03F2
:10101000B0917C030097A105B10551F1E0917D03EA
:10102000F0917E03808190917F0389278083809156
:10103000790390917A03A0917B03B0917C031816F9
:1010400019061A061B06C4F48091790390917A035D
:10105000A0917B03B0917C030197A109B109809312
:10106000790390937A03A0937B03B0937C0304C02D
:101070008091A5010E94DA07FF91EF91BF91AF9196
:101080009F918F917F916F915F914F913F912F91A0
:101090000F900FBE0F901F9018952F923F925F9266
:1010A0006F927F928F929F92AF92BF92CF92DF9278
:1010B000EF92FF920F931F93DF93CF9300D000D056
:1010C000CDB7DEB7A82F1B0129833A834B835C83FE
:1010D0008091A5018A1721F4E8E6F0E0549082C0DF
:1010E0008F3F09F0D9C1A093A501E8E6F0E0549044
:1010F0002FEF521609F4D0C181E0581639F192E071
:10110000591609F449C0552009F06CC014BC15BC2F
:1011100084B5826084BD85B5816085BD2A2F30E0AD
:10112000F901E957FF4FE491F0E0EE0FFF1FED5892
:10113000FF4F859194919093700380936F03255690
:101140003F4FF9018491809371034EC0109280004B
:10115000109281008091810088608093810080914D
:1011600081008160809381002A2F30E0F901E957E6
:10117000FF4FE491F0E0EE0FFF1FED58FF4F859118
:101180009491909377038093760325563F4FF9010E
:1011900084918093780328C01092B0001092B1001F
:1011A0008091B00082608093B0008091B100816036
:1011B0008093B1002A2F30E0F901E957FF4FE49105
:1011C000F0E0EE0FFF1FED58FF4F85919491909343
:1011D0007E0380937D0325563F4FF90184918093D0
:1011E0007F0302C057FC58C18A2F61E00E9421157D
:1011F000552021F0F2E05F1609F0BDC031018824CE
:10120000992460E079E08DE390E0A40193010E94CD
:101210005F2159016A01860175010894E108F1080E
:10122000010911092FEFE216F1040105110509F07A
:1012300008F498C060E271EA87E090E0A4019301AD
:101240000E945F2179018A010894E108F1080109EF
:10125000110982E05816C1F49FEFE916F104010567
:10126000110509F008F483C068E478EE81E090E0AD
:10127000A40193010E945F2179018A010894E10889
:10128000F1080109110983E0AFEFEA16F104010545
:10129000110509F008F467C064E274EF80E090E0A3
:1012A000A40193010E945F2179018A010894E10859
:1012B000F10801091109552011F483E01DC0B2E0C5
:1012C0005B1611F084E018C0EFEFEE16F104010593
:1012D000110509F008F4DEC062E17AE780E090E0F1
:1012E000A40193010E945F2179018A010894E10819
:1012F000F1080109110985E0FFEFEF16F10401057E
:10130000110589F180F169E07DE380E090E0A401BE
:1013100093010E945F2179018A010894E108F10894
:1013200001091109552011F086E001C084E02FEF7A
:10133000E216F10401051105B1F0A8F0860175016E
:101340009AE016950795F794E7949A95D1F7089443
:10135000E108F10801091109552011F087E008C0E2
:1013600085E003C081E0552019F485BD3AC082E0D4
:101370008093B10036C05101CC24DD2460E079E0D7
:101380008DE390E0A60195010E945F2179018A0119
:101390000894E108F1080109110980E0E81680E0ED
:1013A000F80681E0080780E0180710F491E010C00B
:1013B00064E274EF80E090E0A60195010E945F2155
:1013C00079018A010894E108F1080109110993E003
:1013D000A1E05A1631F480918100887F982B909378
:1013E000810089819A81AB81BC810097A105B105FB
:1013F00029F48FEF9FEFAFEFBFEF13C0220C331C28
:10140000B10180E090E029813A814B815C810E94AA
:10141000402128EE33E040E050E00E945F21C90106
:10142000DA01E1E05E16A1F0F2E05F1619F1552055
:1014300099F5E7BC80936B0390936C03A0936D03C5
:10144000B0936E0380916E00826080936E0024C022
:10145000F0928900E0928800809372039093730366
:10146000A0937403B093750380916F0082608093A2
:101470006F0012C0E092B3008093790390937A03D7
:10148000A0937B03B0937C03809170008260809373
:10149000700002C084E06CCF0F900F900F900F90FF
:1014A000CF91DF911F910F91FF90EF90DF90CF9040
:1014B000BF90AF909F908F907F906F905F903F9084
:1014C0002F900895823000F5E82FF0E0EE0FFF1F17
:1014D000E058FC4F71836083882319F08130A1F4B8
:1014E00008C0809169008C7F842B80936900E89A02
:1014F000089580916900440F551F440F551F837F45
:10150000842B80936900E99A0895823080F48823BF
:1015100019F0813021F402C0E89801C0E998E82F61
:10152000F0E0EE0FFF1FE058FC4F1182108208958B
:101530001F920F920FB60F9211242F933F934F9348
:101540005F936F937F938F939F93AF93BF93EF932B
:10155000FF938091800390918103892B29F0E09182
:101560008003F09181030995FF91EF91BF91AF91B5
:101570009F918F917F916F915F914F913F912F91AB
:101580000F900FBE0F901F9018951F920F920FB6DD
:101590000F9211242F933F934F935F936F937F93F9
:1015A0008F939F93AF93BF93EF93FF9380918203A9
:1015B00090918303892B29F0E0918203F0918303BA
:1015C0000995FF91EF91BF91AF919F918F917F917D
:1015D0006F915F914F913F912F910F900FBE0F90A0
:1015E0001F9018952F923F924F925F926F927F9229
:1015F0008F929F92AF92BF92CF92DF92EF92FF9223
:101600000F931F93DF93CF93CDB7DEB73B014C0110
:1016100019012A016D897E898F89988D6A197B0944
:101620008C099D09621A730A840A950AA401930120
:101630000E944021E218F30804091509A801970146
:101640000E9481212A0D3B1D4C1D5D1DB901CA015F
:10165000CF91DF911F910F91FF90EF90DF90CF908E
:10166000BF90AF909F908F907F906F905F904F90C2
:101670003F902F900895089570E0382F20E0622B5E
:10168000732BCB010895EF92FF920F931F937B0171
:101690008C01611571058105910529F420E030E088
:1016A00040E050E00BC00E943123A80197010E9446
:1016B0008121AC01CB01DA019C01AD01B901CA0164
:1016C0001F910F91FF90EF900895EF92FF920F936B
:1016D0001F937B018C01621773078407950764F4DD
:1016E000261B370B480B590BCA01B9010E94430B4B
:1016F000E60EF71E081F191FB701C8011F910F91B1
:10170000FF90EF900895009729F0BC0180E090E0F1
:101710000E9436230895FC010190F081E02DE60F30
:10172000F71F80810895DC01ED91FC9111973097AE
:1017300051F014968D919C9115976817790718F4BC
:10174000E60FF71F40830895FC019B01848195817A
:101750006817790728F4608171816115710529F492
:101760001092840364E873E002C0620F731FCB0120
:101770000895FC010190F081E02DE60FF71F8081B4
:101780000895FC01808191810E940D2408950F939A
:101790001F93CF93DF93FC018B0141155105A1F0FD
:1017A0006115710589F084819581EA0121978C1773
:1017B0009D0708F4EC0160817181C801AE010E94AF
:1017C0008924C00FD11F1882DF91CF911F910F91F3
:1017D00008950F931F93CF93DF93FC018B01411565
:1017E0005105A1F06115710589F084819581EA01A7
:1017F00021978C179D0708F4EC0160817181C80165
:10180000AE010E948924C00FD11F1882DF91CF91B1
:101810001F910F9108950F931F938C01FC018081FC
:1018200091810E948622F80113821282158214820D
:101830001F910F910895FC01DB0114962D913C91AD
:10184000159784819581821B930B8417950710F45B
:1018500080E00895808191816D917C91840F951F26
:10186000A9010E947B249C0180E0232B09F481E0E4
:101870000895FC01DB012481358114968D919C91A2
:1018800015972817390710F480E00895CF0140E03C
:1018900050E00E941B0C0895DF92EF92FF920F938D
:1018A0001F93CF93DF93EC018C819D8148175907DB
:1018B000C8F47A010894E11CF11CE881F981EE0D6D
:1018C000FF1DD080108208811981772767FD7095F0
:1018D000C8010E9498249C010E0D1F1DF801D082A2
:1018E000009719F4EFEFFFEF05C088819981F901A6
:1018F000E81BF90BCF01DF91CF911F910F91FF9062
:10190000EF90DF900895FC01448155814150504093
:101910000E944C0C0895CF93DF93FC01DB0184817E
:1019200095814817590760F4C081D1816D917C91F0
:10193000CE01840F951F0E94A3249C01009719F4E7
:101940002FEF3FEF02C02C1B3D0BC901DF91CF9160
:10195000089540E050E00E948B0C0895CF93DF93F0
:10196000FC01848195814817590768F4C081D181B1
:10197000772767FD7095CE01840F951F0E94602424
:101980009C01009719F42FEF3FEF02C02C1B3D0B79
:10199000C901DF91CF91089540E050E00E94AE0C64
:1019A0000895DC01FB0114962D913C9115978481DB
:1019B00095812817390711F080E0089560817181C1
:1019C0008D919C910E946B249C0180E0232B09F453
:1019D00081E00895FC01DB012481358114968D910D
:1019E0009C9115972817390710F480E00895281B5B
:1019F000390B808191816D917C91820F931F0E94A0
:101A00006B249C0180E0232B09F481E00895DC0124
:101A1000FB01608171818D919C910E946B24292F23
:101A2000332727FD3095209530952227330F221F2D
:101A30003327C9010895DC01FB01608171818D911B
:101A40009C910E946B2440E050E01816190614F097
:101A500041E050E0CA010895DC01FB016081718121
:101A60008D919C910E946B2440E050E0181619065D
:101A700014F441E050E0CA010895DC01FB016081EB
:101A800071818D919C910E946B24292F332727FD12
:101A900030952227330F221F3327C9010895DC0117
:101AA000FB0114962D913C911597848195812817FF
:101AB000390751F4608171818D919C910E946B2452
:101AC0009C0180E0232B09F081E090E00895DC0187
:101AD000FB0114962D913C911597848195812817CF
:101AE000390711F080E00BC0608171818D919C916C
:101AF0000E946B249C0180E0232B09F481E090E09C
:101B00000895FC01DB016D917C91808191810E949F
:101B10006B2408950F931F93CF93DF93EC018B01F8
:101B2000FB01648175818C819D81680F791F7D83A4
:101B30006C838A819B8186179707B8F46F5F7F4F0C
:101B4000888199810E943F234C815D81009729F013
:101B5000998388835B834A8308C0F80184819581D7
:101B6000481B590B5D834C8307C0F801608171816C
:101B7000888199810E945524CE01DF91CF911F91D8
:101B80000F9108950E948A0D0895CF93DF93EC0181
:101B9000CB017B836A8301960E94D9219983888334
:101BA000009721F41B821A821D821C82DF91CF9143
:101BB00008950F931F93CF93DF93EC018B0186174A
:101BC000970709F1FB01248135818C819D81821762
:101BD000930750F4888199810E948622F8016481DC
:101BE0007581CE010E94C50D2881398121153105ED
:101BF00051F0F801848195819D838C83608171818E
:101C0000C9010E947424CE01DF91CF911F910F91E1
:101C100008951F93CF93DF93EC01162F81E090E09E
:101C20009D838C83CE0161E070E00E94C50DE88148
:101C3000F981309721F01083E881F9811182DF91D9
:101C4000CF911F9108951F93CF93DF93EC01162F2F
:101C500081E090E09D838C83CE0161E070E00E9482
:101C6000C50DE881F981309721F01083E881F98171
:101C70001182DF91CF911F9108951F93CF93DF932E
:101C8000EC01162F81E090E09D838C83CE0161E012
:101C900070E00E94C50DE881F981309721F0108332
:101CA000E881F9811182DF91CF911F9108951F93EF
:101CB000CF93DF93EC01162F81E090E09D838C831E
:101CC000CE0161E070E00E94C50DE881F981309796
:101CD00021F01083E881F9811182DF91CF911F916A
:101CE00008950F931F93CF93DF938C01EB016C81C9
:101CF0007D81FC01758364830E94C50DF80180819C
:101D00009181009721F0688179810E947424DF918C
:101D1000CF911F910F9108950F931F93CF93DF934E
:101D20008C01EB016C817D81FC01758364830E94D1
:101D3000C50DF80180819181009721F0688179813A
:101D40000E947424DF91CF911F910F910895EF921B
:101D5000FF920F931F93DF93CF93CDB7DEB7A19779
:101D60000FB6F894DEBF0FBECDBF8C01CB01BA0118
:101D70007E010894E11CF11CA7012AE030E00E94DA
:101D80002725F70101900020E9F73197EE19FF09A7
:101D9000D8011596FC93EE931497C801BF010E94D9
:101DA000C50DF80180819181009719F0B7010E945B
:101DB0007424A1960FB6F894DEBF0FBECDBFCF91AD
:101DC000DF911F910F91FF90EF900895EF92FF9296
:101DD0000F931F93DF93CF93CDB7DEB7A1970FB6C5
:101DE000F894DEBF0FBECDBF8C01CB01BA017E01DE
:101DF0000894E11CF11CA7012AE030E00E9427258D
:101E0000F70101900020E9F73197EE19FF09D80199
:101E10001596FC93EE931497C801BF010E94C50D5F
:101E2000F80180819181009719F0B7010E94742414
:101E3000A1960FB6F894DEBF0FBECDBFCF91DF9154
:101E40001F910F91FF90EF900895EF92FF920F93E3
:101E50001F93DF93CF93CDB7DEB7A1970FB6F8945A
:101E6000DEBF0FBECDBF8C019A0180E090E07E0105
:101E70000894E11CF11CA7010E942725F70101909D
:101E80000020E9F73197EE19FF09D8011596FC9368
:101E9000EE931497C801BF010E94C50DF80180811F
:101EA0009181009719F0B7010E947424A1960FB692
:101EB000F894DEBF0FBECDBFCF91DF911F910F9180
:101EC000FF90EF900895EF92FF920F931F93DF938F
:101ED000CF93CDB7DEB7A1970FB6F894DEBF0FBE94
:101EE000CDBF8C019A0180E090E07E010894E11C56
:101EF000F11CA7010E942725F70101900020E9F7B6
:101F00003197EE19FF09D8011596FC93EE931497BB
:101F1000C801BF010E94C50DF80180819181009721
:101F200019F0B7010E947424A1960FB6F894DEBF91
:101F30000FBECDBFCF91DF911F910F91FF90EF901A
:101F400008950F931F93CF93DF938C01EB016115DD
:101F5000710511F4C6EAD1E0FE0101900020E9F715
:101F60003197EC1BFD0BD8011596FC93EE9314975B
:101F7000C801BF010E94C50DF801808191810097C1
:101F800019F0BE010E947424DF91CF911F910F912F
:101F90000895AF92BF92CF92DF92EF92FF920F938C
:101FA0001F93CF93DF93B82EA92E6B01C82FD92F83
:101FB000FB0160817181CE010E94A10FEE24FF24FC
:101FC00010C0088119810E0D1F1DF801808199270D
:101FD00087FD90950E944424F80180830894E11CB9
:101FE000F11CF60184819581E816F90650F38B2DDA
:101FF0009A2DDF91CF911F910F91FF90EF90DF907D
:10200000CF90BF90AF900895AF92BF92CF92DF92E2
:10201000EF92FF920F931F93CF93DF93B82EA92EC9
:102020006B01C82FD92FFB0160817181CE010E9405
:10203000A10FEE24FF2410C0088119810E0D1F1D71
:10204000F8018081992787FD90950E943C24F80132
:1020500080830894E11CF11CF60184819581E816C7
:10206000F90650F38B2D9A2DDF91CF911F910F918F
:10207000FF90EF90DF90CF90BF90AF900895EF92D8
:10208000FF920F931F93DF93CF93CDB7DEB72C97BB
:102090000FB6F894DEBF0FBECDBFFC017B018617E3
:1020A000970711F401E029C024813581DB011496E2
:1020B0008D919C9115972817390711F000E01DC0EC
:1020C000CE010196BF010E94041009811A81CE0140
:1020D0000796B7010E9404106F817885C8010E949D
:1020E0006B2400E0009709F401E0CE0107960E94FE
:1020F0000B0CCE0101960E940B0C802F2C960FB674
:10210000F894DEBF0FBECDBFCF91DF911F910F912D
:10211000FF90EF900895CF92DF92EF92FF921F937E
:10212000CF93DF936C017B01B9012417350710F4BD
:10213000BA01A901D70114968D919C911597EB01D5
:102140008617970708F4EC01D701ED91FC911197E0
:10215000EC0FFD1F108110826D917C91640F751F33
:10216000C6010E94A10FD701ED91FC91EC0FFD1F5C
:102170001083C601DF91CF911F91FF90EF90DF9008
:10218000CF9008950F931F938C01FB01248135811B
:102190000E948B10C8011F910F9108958F929F92FA
:1021A000AF92BF92CF92DF92EF92FF920F931F9365
:1021B000DF93CF9300D000D000D0CDB7DEB75C0165
:1021C0006B01DB0114968D919C9115970097A1F1FD
:1021D00001974817590780F1F501848195814817C7
:1021E000590750F5ED91FC9100817A014E01089458
:1021F000811C911C1FC0D501ED91FC91EE0DFF1DBE
:1022000080818017A1F4F601248135812E0D3F1DB8
:10221000C401B501A7010E948B10C401B6010E9440
:10222000D10C182FC4010E940B0C112341F4089407
:10223000E108F108F7FEDFCFEE24EA94FE2CC70197
:1022400026960FB6F894DEBF0FBECDBFCF91DF91BB
:102250001F910F91FF90EF90DF90CF90BF90AF90C4
:102260009F908F900895FC01DB0144815581149665
:102270008D919C911597481B590BCF010E94CE1050
:102280000895AF92BF92CF92DF92EF92FF920F9399
:102290001F93DF93CF9300D000D000D0CDB7DEB72F
:1022A0005C018B01DB016D917C916115710521F45D
:1022B000B8010E94710E42C0CE0101960E94A10F8A
:1022C000F801E480F580CC24DD2410C0D801ED9124
:1022D000FC91EC0DFD1D8081992787FD90950E9452
:1022E0003424892B31F00894C11CD11CCE14DF0496
:1022F00068F3ED80FE800DC0D801ED91FC91EE0DEC
:10230000FF1D8081992787FD90950E943424892B99
:1023100031F00894E108F108CE14DF0468F3089462
:10232000E11CF11CC5018E010F5F1F4FB801A60112
:1023300097010E948B10C8010E940B0CC5012696C4
:102340000FB6F894DEBF0FBECDBFCF91DF911F91C6
:102350000F91FF90EF90DF90CF90BF90AF900895D6
:102360002F923F924F925F926F927F928F929F92A5
:10237000AF92BF92CF92DF92EF92FF920F931F9393
:10238000DF93CF93CDB7DEB768970FB6F894DEBF73
:102390000FBECDBF3C01FB012A0119016081718193
:1023A0006115710521F4BF010E94710E5AC07E01B2
:1023B0000894E11CF11CC7010E94A10F8E01095F66
:1023C0001F4FC80166EA71E00E94A10FD02EC12EF6
:1023D0003DE0832E912C8C0E9D1E23E1A22EB12C6C
:1023E000AC0EBD1E24C0C401B70140E050E098010E
:1023F0000E948B108D2D9C2DB4010E948A0DC4016A
:102400000E940B0C8D2D9C2DB1010E948A0DF201B2
:1024100044815581400F511FC501B7010E94C21070
:10242000C701B5010E94D90DC5010E940B0CC7015F
:10243000B2010E94A90C8C01FFEF8F3F9F0799F614
:102440008D2D9C2DB7010E948A0DC3016D2D7C2D11
:102450000E94710E8D2D9C2D0E940B0CC7010E94B5
:102460000B0CC30168960FB6F894DEBF0FBECDBF4C
:10247000CF91DF911F910F91FF90EF90DF90CF9060
:10248000BF90AF909F908F907F906F905F904F9094
:102490003F902F900895DF92EF92FF920F931F933A
:1024A000DF93CF9300D000D000D0CDB7DEB77C0152
:1024B000FB01142FD22E608171816115710521F409
:1024C000BF010E94710E1CC0CE0101960E94A10F97
:1024D00089819A81012F112707FD109501C0D082B3
:1024E000B8010E946024FC010097C9F7C7018E0162
:1024F0000F5F1F4FB8010E94710EC8010E940B0CA4
:10250000C70126960FB6F894DEBF0FBECDBFCF91A0
:10251000DF911F910F91FF90EF90DF9008950F933F
:102520001F93CF93DF938C01EB016115710511F4BB
:10253000C6EAD1E0FE0101900020E9F73197EC1BDB
:10254000FD0BD8011596FC93EE931497C801BF01BB
:102550000E94C50DF80180819181009719F0BE019C
:102560000E947424DF91CF911F910F910895EF92F3
:10257000FF920F931F93DF93CF93CDB7DEB7A19751
:102580000FB6F894DEBF0FBECDBF8C01CB01BA01F0
:102590007E010894E11CF11CA7010E94DE24F701D2
:1025A00001900020E9F73197EE19FF09D80115963F
:1025B000FC93EE931497C801BF010E94C50DF8016A
:1025C00080819181009719F0B7010E947424A1962F
:1025D0000FB6F894DEBF0FBECDBFCF91DF911F9134
:1025E0000F91FF90EF900895EF92FF920F931F933A
:1025F000DF93CF93CDB7DEB7A1970FB6F894DEBFC8
:102600000FBECDBF8C01CB01BA017E010894E11C45
:10261000F11CA7010E94DE24F70101900020E9F7D8
:102620003197EE19FF09D8011596FC93EE93149794
:10263000C801BF010E94C50DF801808191810097FA
:1026400019F0B7010E947424A1960FB6F894DEBF6A
:102650000FBECDBFCF91DF911F910F91FF90EF90F3
:102660000895EF92FF920F931F93DF93CF93CDB70F
:10267000DEB7A1970FB6F894DEBF0FBECDBF8C01B9
:10268000CB017E010894E11CF11CB7010E94BD241E
:10269000F70101900020E9F73197EE19FF09D80101
:1026A0001596FC93EE931497C801BF010E94C50DC7
:1026B000F80180819181009719F0B7010E9474247C
:1026C000A1960FB6F894DEBF0FBECDBFCF91DF91BC
:1026D0001F910F91FF90EF900895EF92FF920F934B
:1026E0001F93DF93CF93CDB7DEB7A1970FB6F894C2
:1026F000DEBF0FBECDBF8C01CB017E010894E11C73
:10270000F11CB7010E94BD24F70101900020E9F7F8
:102710003197EE19FF09D8011596FC93EE931497A3
:10272000C801BF010E94C50DF80180819181009709
:1027300019F0B7010E947424A1960FB6F894DEBF79
:102740000FBECDBFCF91DF911F910F91FF90EF9002
:1027500008951F920F920FB60F9211242F933F935B
:102760004F935F936F937F938F939F93AF93BF9399
:102770002091890330918A0340918B0350918C03FF
:1027800070918D03DA01C9010296A11DB11D672F59
:102790006A5F6D3730F06D57DA01C9010396A11DEC
:1027A000B11D60938D038093890390938A03A09356
:1027B0008B03B0938C038091850390918603A09145
:1027C0008703B09188030196A11DB11D80938503F5
:1027D00090938603A0938703B0938803BF91AF9132
:1027E0009F918F917F916F915F914F913F912F9129
:1027F0000F900FBE0F901F9018958FB7F8942091EF
:10280000890330918A0340918B0350918C038FBFD1
:10281000B901CA0108959FB7F894209185033091BA
:102820008603409187035091880386B5A89B06C014
:102830008F3F21F02F5F3F4F4F4F5F4F9FBF542F70
:10284000432F322F2227280F311D411D511D83E0B8
:10285000220F331F441F551F8A95D1F7B901CA01B2
:102860000895EF92FF920F931F93CF93DF937B0115
:102870008C010E940B14EB010EC00E940B146C1B08
:102880007D0B685E7340C8F30894E108F108010904
:102890001109C851DC4FE114F1040105110569F774
:1028A000DF91CF911F910F91FF90EF9008950197C5
:1028B00039F0019729F0880F991F01970197F1F7D7
:1028C0000895789484B5826084BD84B5816084BDA8
:1028D00085B5826085BD85B5816085BDEEE6F0E099
:1028E000808181608083E1E8F0E0108280818260F5
:1028F0008083808181608083E0E8F0E08081816076
:102900008083E1EBF0E0808184608083E0EBF0E0A5
:10291000808181608083EAE7F0E080818460808349
:1029200080818260808380818160808380818068F3
:1029300080831092C10008958093A7010895982F75
:102940008E3008F09E5097708091A7018295880F75
:10295000880F807C892B80937C0080917A00806432
:1029600080937A0080917A0086FDFCCF20917800D8
:1029700040917900942F80E030E0282B392BC90159
:1029800008951F93CF93DF93182FEB0161E00E940E
:102990002115209709F44AC0CF3FD10509F449C059
:1029A000E12FF0E0E155FF4F84918330C1F0843096
:1029B00028F4813051F08230B1F50CC0863019F125
:1029C000873049F1843079F514C084B5806884BDBE
:1029D000C7BD33C084B5806284BDC8BD2EC08091A0
:1029E0008000806880938000D0938900C093880025
:1029F00024C080918000806280938000D0938B00FF
:102A0000C0938A001AC08091B00080688093B000A3
:102A1000C093B30012C08091B00080628093B00078
:102A2000C093B4000AC0C038D1051CF4812F60E007
:102A300002C0812F61E00E947415DF91CF911F9138
:102A40000895482F50E0CA0185569F4FFC012491FC
:102A500049575F4FFA0184918823C1F0E82FF0E0D5
:102A6000EE0FFF1FE759FF4FA591B491662341F484
:102A70009FB7F8948C91209582238C939FBF0895E3
:102A80009FB7F8948C91822B8C939FBF08958330CD
:102A900071F0843028F48130A1F0823021F514C027
:102AA0008630B1F08730D1F08430E9F404C08091F1
:102AB00080008F7703C0809180008F7D809380009D
:102AC000089584B58F7702C084B58F7D84BD089545
:102AD0008091B0008F778093B00008958091B0000E
:102AE0008F7D8093B0000895FF920F931F93F62E71
:102AF000482F50E0CA0181559F4FFC012491CA0123
:102B000085569F4FFC01149149575F4FFA0104917C
:102B10000023D9F0222319F0822F0E944715E02FBD
:102B2000F0E0EE0FFF1FED58FF4FA591B491FF208D
:102B300031F49FB7F8948C911095812304C09FB70E
:102B4000F8948C91812B8C939FBF1F910F91FF90D4
:102B500008950F931F93482F50E0CA0181559F4F4E
:102B6000FC012491CA0185569F4FFC0104914957ED
:102B70005F4FFA011491112319F420E030E015C0E1
:102B8000222319F0822F0E944715812F90E0880F91
:102B9000991F83589F4FFC01A591B4918C9120E01F
:102BA00030E0802311F021E030E0C9011F910F9146
:102BB00008958F929F92AF92BF92CF92DF92EF9241
:102BC000FF920F931F93CF93DF93A82FB0E0CD0117
:102BD00085569F4FFC018490A957BF4FFD01D490AB
:102BE000662311F4992401C0982CCA01B90120E48C
:102BF0003FE140E050E00E94402120E83EE340E019
:102C000050E00E945F2179018A016D2D70E0660F0E
:102C1000771F63587F4FAA24BB246501FB01A59150
:102C2000B4910BC0AE14BF04C006D10609F44FC066
:102C30000894A11CB11CC11CD11C8C918821891540
:102C400089F30CC0AE14BF04C006D10609F43FC01E
:102C50000894A11CB11CC11CD11C03C0FB01A5918F
:102C6000B4918C918821891569F720E030E040E02B
:102C700050E0FB01C591D4910FC0DA01C9018A0D62
:102C80009B1DAC1DBD1D8E159F05A007B107F9F05A
:102C90002F5F3F4F4F4F5F4F88818821891569F320
:102CA000CA01B90128E032E540E050E00E9440212D
:102CB0006058714C8F4F9F4F20E43FE140E050E05F
:102CC0000E945F21C901DA019C01AD0104C020E02E
:102CD00030E040E050E0B901CA01DF91CF911F918F
:102CE0000F91FF90EF90DF90CF90BF90AF909F90AB
:102CF0008F900895BF92CF92DF92EF92FF920F9341
:102D00001F93CF93DF93E82EF62EB42EC7E0D0E0CA
:102D1000022F10E087E0C82ED12CBB2059F4B60159
:102D20006C1B7D0BC80102C0959587956A95E2F7EB
:102D3000BC0107C0B8010C2E02C0759567950A94B6
:102D4000E2F761708E2D0E9474158F2D61E00E9454
:102D500074158F2D60E00E94741521979FEFCF3F6F
:102D6000D907D9F6DF91CF911F910F91FF90EF9086
:102D7000DF90CF90BF900895CF92DF92EF92FF92B5
:102D80000F931F93CF93DF93F82E062FE42E10E0BE
:102D9000C7E0D0E097E0C92ED12C802F61E00E94DF
:102DA0007415EE2061F48F2D0E94A91596012C1B3D
:102DB0003D0B02C0880F991F2A95E2F709C08F2D9D
:102DC0000E94A9150C2E02C0880F991F0A94E2F7E1
:102DD000182B802F60E00E94741521978FEFCF3F52
:102DE000D807D9F6812FDF91CF911F910F91FF90D6
:102DF000EF90DF90CF9008950895089581E080933B
:102E0000D3036093B0031092D1031092D2030895BC
:102E100081E08093D3036093B0031092D1031092AA
:102E2000D20308958091AF039091AE03891B08955A
:102E30009091AE038091AF03981710F080E0089551
:102E4000E92FF0E0E257FC4F80819F5F9093AE0343
:102E50000895AC012091D6033091D7032115310597
:102E6000E1F09091AE038091AF039817B0F090E03D
:102E700008C0FA01EA0FFB1F8081A257BC4F8C9358
:102E80009F5FA92FB0E0A617B7079CF31092AE037F
:102E90006093AF03CB01F90109950895E091D40344
:102EA000F091D503309729F01092D1031092D203FC
:102EB000099508957093D7036093D603089570938E
:102EC000D5036093D40308950895DF93CF930F92B1
:102ED000CDB7DEB769838091D303882389F08091D1
:102EE000D203803290F48091D103E82FF0E0EF54C8
:102EF000FC4F60838F5F8093D1038093D20305C022
:102F0000CE01019661E00E948C180F90CF91DF9165
:102F100008950E9465170895EF92FF920F931F93F3
:102F2000CF93DF937C01042F8091D303882359F042
:102F3000EB0110E005C0C70169910E9465171F5F92
:102F40001017C8F304C0CB01642F0E948C18DF91C6
:102F5000CF911F910F91FF90EF900895DB010D909D
:102F60000020E9F71197A61BB70B4A2F0E948C1778
:102F700008958091B00361EB73E04091D20321E0AA
:102F80000E9449181092D1031092D2031092D303D9
:102F90000895413208F040E2862F6EE873E00E9407
:102FA00012181092AE038093AF0308950E94C917C0
:102FB00008951092AE031092AF031092D1031092B5
:102FC000D2030E94FB1708950F931F938C01862F45
:102FD0000E940E188EE497E10E94AC1889E297E1F6
:102FE0000E94A718C8010E94D9171F910F91089538
:102FF0000E94E41708951092D903449A459AE9EB88
:10300000F0E080818E7F808380818D7F808388E463
:103010008093B80085E48093BC000895880F809366
:10302000BA000895982F413210F040E030C08091EE
:10303000D9038823E1F781E08093D9038FEF809350
:1030400044041092FF034150409300044F5F990FD6
:1030500091609093DA0385EE8093BC008091D90350
:103060008130E1F38091FF03841710F44091FF0356
:1030700020E030E00AC0FB01E20FF31FD901A152AA
:10308000BC4F8C9180832F5F3F4F2417A0F3842F78
:1030900008951F93582F122F413210F081E03AC04B
:1030A0008091D9038823E1F782E08093D9038FEFE1
:1030B000809344041092FF0340930004AFEDB3E00B
:1030C000FB0102C081918D938E2F861B8417D0F354
:1030D000852F90E0880F991F8093DA0385EE809307
:1030E000BC00112321F08091D9038230E1F380915B
:1030F00044048F3F11F480E00DC08091440480327D
:1031000011F482E007C080914404803311F084E020
:1031100001C083E01F910895482F613210F081E0D3
:1031200008958091D903843011F082E0089560936E
:103130002204A1E0B4E0842F9C01F90102C0819136
:103140008D938E2F841B8617D0F380E00895909383
:10315000DE038093DD0308959093DC038093DB030B
:103160000895882311F085EC01C085E88093BC00A8
:10317000089585ED8093BC008091BC0084FDFCCF58
:103180001092D903089585EC8093BC001092D90366
:1031900008951F920F920FB60F9211242F933F9311
:1031A0004F935F936F937F938F939F93AF93BF934F
:1031B000EF93FF938091B90090E0887F9070803604
:1031C000910509F4DCC081369105CCF58832910572
:1031D00009F47BC089329105B4F48031910509F47A
:1031E0006FC0813191053CF4009709F431C1089713
:1031F00009F039C165C08831910509F466C080972E
:1032000009F031C17DC08034910509F49FC081343B
:10321000910544F48033910509F47DC0C89709F005
:1032200022C184C08035910509F484C08835910598
:1032300009F491C08834910509F015C198C0883906
:10324000910509F4FDC089399105ECF488379105A1
:1032500009F495C0893791054CF48836910509F435
:103260008EC08037910509F0FEC089C0883891056D
:1032700009F4E6C08039910509F487C080389105CA
:1032800009F0F1C082C0803B910509F4B0C0813BD8
:1032900091054CF4803A910509F489C0883A91056A
:1032A00009F0E1C0A4C0803C910509F4CDC0883C80
:1032B000910509F4C9C0883B910509F0D4C0ACC0A0
:1032C0008091DA038093BB00B9C09091FF03809195
:1032D0000004981768F49091FF03E92FF0E0E152A1
:1032E000FC4F80818093BB009F5F9093FF03A6C03B
:1032F00085ED8093BC008091BC0084FDFCCFB1C003
:1033000080E28093440485ED8093BC008091BC00F2
:1033100084FDFCCFA6C080E38093440485ED8093B8
:10332000BC008091BC0084FDFCCF9BC088E38093EF
:1033300044048AC08091FF039091BB00E82FF0E025
:10334000E152FC4F90838F5F8093FF039091FF03C6
:103350008091000471C08091FF039091BB00E82F21
:10336000F0E0E152FC4F90838F5F8093FF0385ED87
:103370008093BC008091BC0084FDFCCF72C083E0D0
:103380008093D9031092430459C080914304803242
:1033900008F056C0809143049091BB00E82FF0E004
:1033A000ED5DFB4F90838F5F8093430447C0809116
:1033B0004304803230F4E0914304F0E0ED5DFB4FD4
:1033C000108285ED8093BC008091BC0084FDFCCF11
:1033D0001092D90360914304E091DD03F091DE0384
:1033E00083E294E070E00995109243042DC084E0DC
:1033F0008093D9031092210410922204E091DB0300
:10340000F091DC03099580912204882329F481E05E
:10341000809322041092010490912104E92FF0E09E
:10342000EF5FFB4F80818093BB009F5F90932104EF
:103430009091210480912204981710F485EC01C02A
:1034400085E88093BC000FC085EC8093BC0009C068
:103450001092440485ED8093BC008091BC0084FDF3
:10346000FCCF1092D903FF91EF91BF91AF919F9143
:103470008F917F916F915F914F913F912F910F901D
:103480000FBE0F901F901895EF92FF920F931F930E
:103490007B018C0120E030E040E05FE40E94C01D31
:1034A00088238CF0C801B70120E030E040E05FE401
:1034B0000E94BC1B0E947E1E9B01AC01205030402C
:1034C0004040504806C0C801B7010E947E1E9B01C3
:1034D000AC01B901CA011F910F91FF90EF900895BF
:1034E000A0E0B0E0E6E7FAE10C949C21DC012B01BE
:1034F000FA019C91923008F439C1EB018881823045
:1035000008F433C1943069F4843009F02FC1119666
:103510009C9111978981981709F428C1A8EAB1E014
:1035200025C1843009F421C18230A9F4923009F018
:103530001DC19A01AD0188E0EA010990AE01E901DF
:1035400009929E018150C1F7E201898111969C91F7
:103550008923818308C1923009F407C112962D9006
:103560003C901397EB018A819B811496AD90BD909E
:10357000CD90DC901797EC80FD800E811F8191012A
:10358000281B390BB90137FF04C066277727621B58
:10359000730B603271050CF061C0121613066CF5E6
:1035A00037014801062E04C0969487947794679457
:1035B0000A94D2F721E030E040E050E004C0220F4E
:1035C000331F441F551F6A95D2F7215030404040A9
:1035D00050402E213F214023512321153105410523
:1035E000510521F021E030E040E050E079018A010E
:1035F000E628F728082919293CC0232BD1F1260EEB
:10360000371E35014601062E04C0969487947794A0
:1036100067940A94D2F721E030E040E050E004C023
:10362000220F331F441F551F6A95D2F72150304097
:10363000404050402A213B214C215D21211531057C
:103640004105510521F021E030E040E050E0590112
:103650006A01A628B728C828D9280BC08215930567
:103660002CF01C01AA24BB24650103C0EE24FF2416
:10367000870111969C91D20111968C91981709F4AB
:1036800045C0992339F0A80197012A193B094C0933
:103690005D0906C0A60195012E193F09400B510B8B
:1036A00057FD08C0118233822282248335834683EA
:1036B00057831DC081E08183338222828827992726
:1036C000DC01821B930BA40BB50B84839583A6832B
:1036D000B7830DC0220F331F441F551F248335832A
:1036E00046835783828193810197938382832481C8
:1036F000358146815781DA01C9010197A109B109D4
:103700008F5F9F4FAF4FBF4328F30BC0918333822E
:103710002282EA0CFB1C0C1D1D1DE482F58206832F
:10372000178383E08083248135814681578157FF49
:103730001AC0C901AA2797FDA095BA2F8170907071
:10374000A070B0705695479537952795822B932B8F
:10375000A42BB52B84839583A683B7838281938121
:10376000019693838283DF0101C0D201CD01CDB7E1
:10377000DEB7E2E10C94B821A0E2B0E0E2ECFBE1BC
:103780000C94A82169837A838B839C832D833E8349
:103790004F835887E9E0EE2EF12CEC0EFD1ECE0192
:1037A0000196B7010E946F208E010F5E1F4FCE0160
:1037B0000596B8010E946F208A8991E089278A8B3B
:1037C000C701B801AE01475E5F4F0E94701A0E94A8
:1037D0009A1FA096E6E00C94C421A0E2B0E0E3EFCB
:1037E000FBE10C94A82169837A838B839C832D83CE
:1037F0003E834F835887F9E0EF2EF12CEC0EFD1E2F
:10380000CE010196B7010E946F208E010F5E1F4FFF
:10381000CE010596B8010E946F20C701B801AE0124
:10382000475E5F4F0E94701A0E949A1FA096E6E0C2
:103830000C94C421A0E2B0E0E0E2FCE10C949C21F5
:1038400069837A838B839C832D833E834F83588740
:10385000CE010196BE01675F7F4F0E946F20CE01AF
:103860000596BE016F5E7F4F0E946F209985923052
:1038700088F089898230C8F0943019F4823051F48C
:1038800004C0843029F4923081F488EA91E0C6C003
:10389000923049F420E09A858A89981321E02A879A
:1038A000CE010996BBC0823049F420E09A858A890E
:1038B000981321E02A8BCE014196B0C02D843E841E
:1038C0004F8458886D887E888F88988CEE24FF24DA
:1038D0008701AA24BB24650140E050E060E070E06D
:1038E000E0E0F0E0C10181709070892BE9F0E60C16
:1038F000F71C081D191D9A01AB012A0D3B1D4C1D1B
:103900005D1D80E090E0A0E0B0E0E614F70408055B
:10391000190520F481E090E0A0E0B0E0BA01A9012F
:10392000480F591F6A1F7B1FAA0CBB1CCC1CDD1C37
:1039300097FE08C081E090E0A0E0B0E0A82AB92A94
:10394000CA2ADB2A3196E032F10549F0660C771C71
:10395000881C991C5694479437942794C3CFFA85B2
:10396000EA892B893C898B859C85280F391F2E5F1E
:103970003F4F17C0CA0181709070892B61F0169576
:103980000795F794E79480E090E0A0E0B0E8E82A9B
:10399000F92A0A2B1B2B76956795579547952F5F2C
:1039A0003F4F77FDE7CF0CC0440F551F661F771FB1
:1039B00017FD4160EE0CFF1C001F111F215030400D
:1039C000403090E0590790E0690790E4790760F390
:1039D0002B8F3C8FDB01CA018F779070A070B07085
:1039E00080349105A105B10561F447FD0AC0E114D9
:1039F000F1040105110529F0405C5F4F6F4F7F4FC7
:103A000040781A8EFE1711F081E08A8F4D8F5E8FFD
:103A10006F8F78A383E0898FCE0149960E949A1F09
:103A2000A096E2E10C94B821A8E1B0E0EAE1FDE162
:103A30000C94A42169837A838B839C832D833E839A
:103A40004F835887B9E0EB2EF12CEC0EFD1ECE0112
:103A50000196B7010E946F208E010F5E1F4FCE01AD
:103A60000596B8010E946F202985223008F47EC097
:103A70003989323010F4B8017CC08A859A89892747
:103A80008A87243011F0223031F4231709F06EC0F8
:103A900068EA71E06EC0343039F41D861E861F86D8
:103AA000188A1C861B8604C0323021F484E0898782
:103AB000B7015FC02B853C858B899C89281B390BFE
:103AC0003C872B87ED84FE840F851889AD88BE88DE
:103AD000CF88D88CEA14FB040C051D0540F4EE0CCD
:103AE000FF1C001F111F215030403C872B8720E016
:103AF00030E040E050E080E090E0A0E0B0E460E042
:103B000070E0EA14FB040C051D0540F0282B392B4E
:103B10004A2B5B2BEA18FB080C091D09B695A795E3
:103B200097958795EE0CFF1C001F111F6F5F7F4F4D
:103B30006F31710531F7DA01C9018F779070A0708C
:103B4000B07080349105A105B10561F427FD0AC06C
:103B5000E114F1040105110529F0205C3F4F4F4F9E
:103B60005F4F20782D873E874F87588BBE01675F58
:103B70007F4FCB010E949A1F6896EAE00C94C02107
:103B8000A8E1B0E0E6ECFDE10C94A82169837A831A
:103B90008B839C832D833E834F83588789E0E82E57
:103BA000F12CEC0EFD1ECE010196B7010E946F2094
:103BB0008E010F5E1F4FCE010596B8010E946F2047
:103BC0008985823040F08989823028F0C701B801A8
:103BD0000E94E72001C08FEF6896E6E00C94C421B4
:103BE000A8E1B0E0E6EFFDE10C94A82169837A83B7
:103BF0008B839C832D833E834F83588789E0E82EF7
:103C0000F12CEC0EFD1ECE010196B7010E946F2033
:103C10008E010F5E1F4FCE010596B8010E946F20E6
:103C20008985823040F08989823028F0C701B80147
:103C30000E94E72001C081E06896E6E00C94C42170
:103C4000A8E0B0E0E6E2FEE10C94A5219B01AC0106
:103C500083E08983DA01C9018827B7FD8395992715
:103C6000AA27BB27B82E211531054105510519F4A6
:103C700082E089833AC08823A9F0203080E03807A9
:103C800080E0480780E8580729F460E070E080E0B1
:103C90009FEC30C0EE24FF248701E21AF30A040BE4
:103CA000150B02C079018A018EE1C82ED12CDC826D
:103CB000CB82ED82FE820F831887C801B7010E9474
:103CC0004B1F01971816190684F4082E04C0EE0C39
:103CD000FF1C001F111F0A94D2F7ED82FE820F8392
:103CE0001887C81AD90ADC82CB82BA82CE01019623
:103CF0000E949A1F2896E9E00C94C121ACE0B0E044
:103D0000E4E8FEE10C94AC2169837A838B839C8385
:103D1000CE010196BE016B5F7F4F0E946F208D81A7
:103D2000823061F1823050F1843021F48E81882319
:103D300051F12EC02F81388537FD20C06E812F3183
:103D400031051CF06623F9F023C08EE190E0821B60
:103D5000930B29853A854B855C8504C0569547951C
:103D6000379527958A95D2F76623B1F050954095FF
:103D7000309521953F4F4F4F5F4F0EC020E030E010
:103D800040E050E009C02FEF3FEF4FEF5FE704C086
:103D900020E030E040E050E8B901CA012C96E2E0B2
:103DA0000C94C821A8E0B0E0E8EDFEE10C94A42159
:103DB0007B018C01611571058105910519F482E083
:103DC000898360C083E089838EE1C82ED12CDC8298
:103DD000CB82ED82FE820F831887C801B7010E9453
:103DE0004B1FFC013197F7FF3BC0222733272E1BC7
:103DF0003F0B57016801022E04C0D694C794B794B4
:103E0000A7940A94D2F740E050E060E070E081E0CF
:103E100090E0A0E0B0E004C0880F991FAA1FBB1F6C
:103E20002A95D2F70197A109B1098E219F21A023DC
:103E3000B1230097A105B10521F041E050E060E019
:103E400070E04A295B296C297D294D835E836F834D
:103E500078878EE190E08E1B9F0B9C838B8312C032
:103E6000309781F00E2E04C0EE0CFF1C001F111FB6
:103E70000A94D2F7ED82FE820F831887CE1ADF0AEA
:103E8000DC82CB821A82CE0101960E949A1F28966C
:103E9000EAE00C94C021EF92FF920F931F937B01F5
:103EA0008C0180E0E81680E0F80681E0080780E0F9
:103EB000180788F48FEFE816F1040105110531F0B9
:103EC00028F088E090E0A0E0B0E017C080E090E04B
:103ED000A0E0B0E012C080E0E81680E0F80680E0E4
:103EE000080781E0180728F088E190E0A0E0B0E042
:103EF00004C080E190E0A0E0B0E020E230E040E0EB
:103F000050E0281B390B4A0B5B0B04C01695079534
:103F1000F794E7948A95D2F7F701E055FE4F808138
:103F2000281B310941095109C9011F910F91FF90C7
:103F3000EF900895DF92EF92FF920F931F93FC0191
:103F4000E480F58006811781D1808081823048F439
:103F500080E090E0A0E1B0E0E82AF92A0A2B1B2BD0
:103F6000A5C0843009F49FC0823021F4EE24FF24E0
:103F7000870105C0E114F1040105110519F4E0E021
:103F8000F0E096C0628173819FEF623879070CF090
:103F90005BC022E83FEF261B370B2A3131052CF09E
:103FA00020E030E040E050E02AC0B801A701022E36
:103FB00004C076956795579547950A94D2F781E0A6
:103FC00090E0A0E0B0E004C0880F991FAA1FBB1FBB
:103FD0002A95D2F70197A109B1098E219F21A0232B
:103FE000B1230097A105B10521F081E090E0A0E0A8
:103FF000B0E09A01AB01282B392B4A2B5B2BDA015D
:10400000C9018F779070A070B07080349105A105C0
:10401000B10539F427FF09C0205C3F4F4F4F5F4F78
:1040200004C0215C3F4F4F4F5F4FE0E0F0E0203095
:10403000A0E03A07A0E04A07A0E45A0710F0E1E048
:10404000F0E079018A0127C06038710564F5FB0151
:10405000E158FF4FD801C7018F779070A070B07002
:1040600080349105A105B10539F4E7FE0DC080E467
:1040700090E0A0E0B0E004C08FE390E0A0E0B0E00A
:10408000E80EF91E0A1F1B1F17FF05C0169507959E
:10409000F794E794319687E016950795F794E7949F
:1040A0008A95D1F705C0EE24FF248701EFEFF0E0F9
:1040B0006E2F679566276795902F9F77D794DD249D
:1040C000D7948E2F8695492F462B582F5D29B701FF
:1040D000CA011F910F91FF90EF90DF900895FC01AE
:1040E000DB01408151812281622F6F7770E0221FB6
:1040F0002227221F9381892F880F822B282F30E0BF
:10410000991F9927991F11969C9311972115310595
:10411000A9F5411551056105710511F482E037C01B
:1041200082E89FEF13969C938E9312979A01AB01AE
:1041300067E0220F331F441F551F6A95D1F783E0B4
:104140008C930DC0220F331F441F551F12968D9163
:104150009C911397019713969C938E9312972030FE
:1041600080E0380780E0480780E4580758F3149649
:104170002D933D934D935C93179708952F3F3105F1
:1041800079F4411551056105710519F484E08C93AA
:10419000089564FF03C081E08C9312C01C9210C08C
:1041A0002F57304013963C932E93129783E08C93B5
:1041B00087E0440F551F661F771F8A95D1F77064FB
:1041C00014964D935D936D937C93179708951F9369
:1041D000DC01FB019C91923008F447C08081823061
:1041E00008F443C0943051F411961C91843099F531
:1041F0008181682F70E0611B71093FC0843021F01C
:10420000923031F48230B9F18181882389F12DC057
:1042100011961C9111978230F1F081811817D9F411
:1042200012962D913C911397828193818217930767
:1042300094F028173907BCF014968D919D910D903C
:10424000BC91A02D248135814681578128173907DB
:104250004A075B0718F4112341F00AC0821793073D
:10426000A407B50740F4112319F061E070E005C020
:104270006FEF7FEF02C060E070E0CB011F91089507
:10428000629FD001739FF001829FE00DF11D649F3A
:10429000E00DF11D929FF00D839FF00D749FF00DC6
:1042A000659FF00D9927729FB00DE11DF91F639F67
:1042B000B00DE11DF91FBD01CF0111240895A1E248
:1042C0001A2EAA1BBB1BFD010DC0AA1FBB1FEE1F90
:1042D000FF1FA217B307E407F50720F0A21BB30BDB
:1042E000E40BF50B661F771F881F991F1A9469F757
:1042F00060957095809590959B01AC01BD01CF01B3
:10430000089597FB092E05260ED057FD04D0D7DF60
:104310000AD0001C38F450954095309521953F4FB8
:104320004F4F5F4F0895F6F7909580957095619582
:104330007F4F8F4F9F4F08952F923F924F925F92E2
:104340006F927F928F929F92AF92BF92CF92DF92A5
:10435000EF92FF920F931F93CF93DF93CDB7DEB70A
:10436000CA1BDB0B0FB6F894DEBF0FBECDBF09949E
:104370002A88398848885F846E847D848C849B84F5
:10438000AA84B984C884DF80EE80FD800C811B8103
:10439000AA81B981CE0FD11D0FB6F894DEBF0FBE32
:1043A000CDBFED010895EE0FFF1F0590F491E02DB4
:1043B0000994CF93DF93BC018230910510F462E041
:1043C00070E0A0914704B0914804ED01E0E0F0E016
:1043D00040E050E021C0888199818617970769F4F1
:1043E0008A819B81309719F09383828304C09093D4
:1043F000480480934704FE0134C06817790738F4F5
:104400004115510519F08417950708F4AC01FE0118
:104410008A819B819C01E9012097E9F641155105AC
:10442000A9F1CA01861B970B049708F4BA01E0E0D2
:10443000F0E02AC08D919C91119784179507F9F4AB
:104440006417750781F412968D919C91139730979C
:1044500019F09383828304C09093480480934704A7
:10446000FD0132964FC0CA01861B970BFD01E80F74
:10447000F91F6193719302978D939C9343C0FD0143
:10448000828193819C01D9011097A1F68091450406
:1044900090914604892B41F48091B2029091B3022D
:1044A00090934604809345044091B4025091B50224
:1044B0004115510541F44DB75EB78091B00290911E
:1044C000B102481B590B2091450430914604241732
:1044D0003507B0F4CA01821B930B8617970780F04B
:1044E000AB014E5F5F4F8417950750F0420F531F8B
:1044F0005093460440934504F9016193719302C0BF
:10450000E0E0F0E0CF01DF91CF910895CF93DF930A
:10451000009709F450C0EC0122971B821A82A091E7
:104520004704B0914804109709F140E050E0AC17FF
:10453000BD0708F1BB83AA83FE0121913191E20FEF
:10454000F31FAE17BF0779F48D919C911197280F37
:10455000391F2E5F3F4F3983288312968D919C918E
:1045600013979B838A834115510571F4D0934804B6
:10457000C093470420C012968D919C911397AD0172
:10458000009711F0DC01D3CFFA01D383C2832191CC
:104590003191E20FF31FCE17DF0769F4888199810B
:1045A000280F391F2E5F3F4FFA01318320838A8104
:1045B0009B8193838283DF91CF910895A0E0B0E047
:1045C000E4EEF2E20C94A421EC01A880B980CA8048
:1045D000DB80A114B104C104D10441F484E2A82E0B
:1045E00089EDB82E8BE5C82E87E0D82EC601B5011F
:1045F0002DE133EF41E050E00E94812127EA31E4D0
:1046000040E050E00E9440217B018C01C601B501D1
:104610002DE133EF41E050E00E948121CA01B90150
:104620002CEE34EF4FEF5FEF0E9440216E0D7F1DA7
:10463000801F911F97FF04C06150704080409048D8
:10464000688379838A839B839B01AC015F77B9017F
:10465000CA01CDB7DEB7EAE00C94C0210E94DE2289
:10466000089586EB92E00E94DE2208956093B602E0
:104670007093B7028093B8029093B9020895A0E0B6
:10468000B0E0E5E4F3E20C94A2218C01009729F458
:10469000CB010E94D9218C01BAC09EEFE92E9FEF79
:1046A000F92EE00EF11E5801A60EB71EAE14BF047F
:1046B00008F4ABC08EEF882E8FEF982E8A0C9B1CCF
:1046C000E7014881598146175707B8F04530510531
:1046D00008F49DC0CA0104978617970708F497C08D
:1046E00042505040461B570BF4015183408379835D
:1046F0006883C5010E9486228AC06B01C41AD50A4C
:10470000E0914704F0914804A0E0B0E0C0E0D0E0C0
:1047100042C0E815F905A1F5208131812C153D0530
:1047200078F1C90102968C159D05A8F04E5F5F4F88
:10473000420F531FE7015983488322813381109729
:1047400029F013963C932E93129761C0309348043E
:10475000209347045CC0225030402C193D0931831E
:104760002083109729F01396FC93EE93129704C0C0
:10477000F0934804E0934704F7017183608347C0D6
:1047800080819181C817D90708F4EC01DF0182818B
:1047900093819C01F901309709F0BBCF400F511F65
:1047A000809145049091460484179507E9F4C61753
:1047B000D707D0F42091B4023091B502211531050C
:1047C00041F42DB73EB78091B0029091B102281B01
:1047D000390BA216B306C8F4B0924604A092450461
:1047E000E7017983688313C0CB010E94D921EC01D2
:1047F000009759F0F70140815181B8010E944C2483
:10480000C8010E9486228E0102C000E010E0C801AB
:10481000CDB7DEB7ECE00C94BE211F93FC019927C5
:104820008827BC01E89411911032E9F3193010F097
:104830001E30C8F31B3251F01D3249F4689406C093
:104840000E941225610F711D811D911D1191105340
:104850001A30B0F33EF490958095709561957F4F36
:104860008F4F9F4F1F910895911116C1803219F0FB
:1048700089508550D0F708959111089581548A5137
:1048800008F4805E855A08959111089581568A51E1
:1048900008F4805285580895FB01DC0102C00190A4
:1048A0000D9241505040D8F70895FB01DC010D9066
:1048B0000020E9F7119701900D920020E1F708958B
:1048C000FC018191861721F08823D9F79927089553
:1048D0003197CF010895FB01DC018D910190801982
:1048E0000110D9F3990B0895FB01DC0101900D92A1
:1048F0000020E1F70895FB01DC014150504030F009
:104900008D910190801919F40020B9F7881B990B3B
:104910000895FB01DC014150504048F001900D9298
:104920000020C9F701C01D9241505040E0F70895A2
:10493000FC0181E090E00190061609F4CF0100200F
:10494000D1F701970895FB0151915523A9F0BF01BB
:10495000DC014D9145174111E1F759F4CD0101906A
:10496000002049F04D9140154111C9F3FB0141115F
:10497000EFCF81E090E001970895FB019F01E8945B
:104980004230C4F04532B4F44A3029F497FB1EF4A7
:10499000909581959F4F642F77270E945F25805DBA
:1049A0008A330CF0895D8193CB010097A1F716F44F
:1049B0005DE251931082C9010C944F25FA01CF9307
:1049C000FF93EF93223044F1253234F5C22FE8945F
:1049D000CA3049F497FB3EF49095809570956195A7
:1049E0007F4F8F4F9F4F2C2F332744275527FF93FF
:1049F000EF930E945F21EF91FF91605D6A330CF0AD
:104A0000695D6193B901CA01605070408040904077
:104A100051F716F4CDE2C19310828F919F91CF91FF
:104A20000C944F25592F482F372F262F660F771FAD
:104A3000881F991F660F771F881F991F620F731FAA
:104A4000841F951F660F771F881F991F0895FA010D
:104A5000CF93FF93EF932230CCF02532BCF4C22FDA
:104A60002C2F332744275527FF93EF930E945F2174
:104A7000EF91FF91605D6A330CF0695D6193B9015C
:104A8000CA01605070408040904051F710828F9171
:104A90009F91CF910C944F25992788270895DC0189
:104AA000FC01672F71917723E1F7329704C07C9165
:104AB0006D9370836291AE17BF07C8F30895AA1B68
:104AC000BB1B51E107C0AA1FBB1FA617B70710F0F9
:104AD000A61BB70B881F991F5A95A9F7809590952B
:0A4AE000BC01CD010895F894FFCF4A
:104AEA000D0A2B494E513D310D0A000D0A2B535424
:104AFA00574D4F443D300D0A000D0A2B53544E4179
:104B0A003D4164617074696373456C65637469637C
:104B1A000D0A000D0A2B53544F4155543D310D0ACD
:104B2A00000D0A2B53544155544F3D300D0A000DC8
:104B3A000A202B535450494E3D303030300D0A0074
:104B4A000D0A2B4C4F53535245434F4E4E3D300D99
:104B5A000A0007F000000000009304E004F804389B
:104B6A000463044904870400000000DB00E004F841
:104B7A0004DB00DB00DB00DB002E0000000000DBB2
:104B8A0000E004F804FF000100000000000000003B
:104B9A0000010202030303030404040404040404DA
:104BAA0005050505050505050505050505050505AB
:104BBA00060606060606060606060606060606068B
:104BCA00060606060606060606060606060606067B
:104BDA00070707070707070707070707070707075B
:104BEA00070707070707070707070707070707074B
:104BFA00070707070707070707070707070707073B
:104C0A00070707070707070707070707070707072A
:104C1A00080808080808080808080808080808080A
:104C2A0008080808080808080808080808080808FA
:104C3A0008080808080808080808080808080808EA
:104C4A0008080808080808080808080808080808DA
:104C5A0008080808080808080808080808080808CA
:104C6A0008080808080808080808080808080808BA
:104C7A0008080808080808080808080808080808AA
:104C8A00080808080808080808080808080808089A
:0A4C9A0020004904000001000000A2
:00000001FF
